:200000000EC0189518951895189518951895189518951895189518958FC0189518950FE506
:200020000DBF02E00EBF00E806BD00E006BD379887D009E007BBC498C39A16E12BD0C39820
:200040001CD01ED0B13024F4AA2311F029D000C001E00F9372D000E205BF78948895F89426
:2000600000E005BF0F910A95A1F701D0E5CFC09ABFEFAFEF12D0C0980895B49BFECF08954A
:20008000BB27AA271196B13024F418E903D0B499F9CF08951A95F1F708951197F1F7089526
:2000A000CFEF62D0C22FC39500EC0C1710F411D0CC272C2FCFEF4DD0C22FDF9712F0959755
:2000C00012F4AA27BB27BB2309F0AFEF2A2F41D00895CDEF49D0F22F47D0E22FDD27CC27D6
:2000E00033E0FF93EF9303E007BFE895EE27FF2701E107BFE89540E437D0022E35D0122EB3
:2001000001E007BFE895E395E3954A95A9F7EF91FF9105E007BFE895FF9631963A9509F7E9
:200120000FE00F1710F4F2E0EE27CDEF2F2F11D0C3952E2F0ED00895189509E601BD08959D
:20014000A89500E004BF01B5086101BD00E001BD0895DD27E199FDCF00E00CBBDFBBCEBB93
:200160002DBBE29AE19A0895DD27E199FDCFDFBBCEBBE09A2DB3C3950895FFFFFFFFFFFF4D
:20018000FFFFFFFFFFFFFFFFFFFFFFFFFFFFFFFFFFFFFFFFFFFFFFFFFFFFFFFFFFFFFFFF7F
:2001A000FFFFFFFFFFFFFFFFFFFFFFFFFFFFFFFFFFFFFFFFFFFFFFFFFFFFFFFFFFFFFFFF5F
:2001C000FFFFFFFFFFFFFFFFFFFFFFFFFFFFFFFFFFFFFFFFFFFFFFFFFFFFFFFFFFFFFFFF3F
:2001E000FFFFFFFFFFFFFFFFFFFFFFFFFFFFFFFFFFFFFFFFFFFFFFFFFFFFFFFFFFFFFFFF1F
:200200006C6174006A64666A68666064666868646600684500460042404340414043604011
:20022000426343434440434264406360634465644160416460666264646365676100446247
:20024000676165646927262666626564006062204624262020002026262020262220212693
:200260002021242022230067666666676667666766666767666667656867666666000040A7
:200280006C6174006A64666A68666064666868646600684500460042404340414043604091
:2002A0004263434344404342644063606344656441604164606662646463656761004462C7
:2002C00068686061606850707850535053545050530000000000000000007778507770706A
:2002E000787777777077777870710070777700707777707071787770787077707778707759
:2003000071606868713736286070616528607220503528303032313626313026323031366A
:20032000203130123033787878780078797778787778777878777A777877777A000240406F
:200340006868606160685070785053505354505053000000000000000000777850777070E9
:200360007877777770777778707100707777007077777070717877707870777077787077D8
:20038000707070707077717600707776777078707778707777777176707077717170767267
:2003A0007077767877707076777770707878707076707677717870707776767176707670C1
:2003C00070606565713636286600000000000000000000000000000000000026323030322E
:2003E0002030353232327879787676777776777676777676777676777776777677000040F8
:200400007070707070777176007077767770787077787077777771767070777171707672E6
:20042000707776787770707677777070787870707670767771787070777676717670767040
:2004400077707076767876707276737670767677776670767076777570767071767072752E
:200460007476707076006672767574767670707277700072777678787170767170777076FC
:20048000766065687837302660006065266670205634263030323124283030263230303666
:2004A00020303032323378786E7677767678777677787776767776767778787778044040FA
:2004C0007770707676787670727673767076767777667076707677757076707176707275AE
:2004E00074767070760066727675747676707072777000727776787871707671707770767C
:20050000767070706800717076706470746471707676767878767676707072767678767108
:200520000070767578767675717777687776777676757074767776767076667076657776BA
:20054000766169687037362660706565266672205630263130383136263130262230313626
:200560002031353232327979797678777900007777776D76777879777A7776767704004057
:20058000767070706800717076706470746471707676767878767676707072767678767188
:2005A00000707675787676757177776877767776767570747677767670766670766577763A
:2005C0007070707070727876787070777778707876777070707877717770767770777771A5
:2005E000767770777070777076767071707876767676777777717770717071707077707687
:200600007061656571303626667260652666702056302630303231302A3030263230313671
:20062000203135323033777878767778787779767877777778777877777778777800404065
:20064000707070707072787678707077777870787677707070787771777076777077777124
:20066000767770777070777076767071707876767676777777717770717071707077707606
:20068000707770707470767000767070707876777676777770777770707078707676777655
:2006A0007670707070727776707070707670767278707670787777707371787670767674D1
:2006C0007561656471303424647065642464722054342430303030362430302430303134BC
:2006E000203135303231777575757976747475777574757675757575757574757506004012
:200700007077707074707670007670707078767776767777707777707070787076767776D4
:20072000767070707072777670707070767076727870767078777770737178767076767450
:20074000757475757474767574747674757676757076717676747675747574757676747502
:200760007676767775757475767075747776747676757470757074747676717476767474E6
:200780007660646571363624667264642466702050302430303031342430302430303136F7
:2007A00020303530303175757676757676767576757675757676767577757574770640400D
:2007C000757475757474767574747674757676757076717676747675747574757676747582
:2007E000767676777575747576707574777674767675747075707474767671747676747466
:200800007574717574767676747575757674757175787465647470776465747675666565B3
:20082000676564656874747474707476747676767674767676747670747476707075747579
:20084000656065647935362866706064266672205634243030303036243130243030303435
:200860002031343232327577767776766D756D757776006E6D75767676756F75760800401E
:20088000757471757476767674757575767475717578746564747077646574767566656533
:2008A0006765646568747474747074767476767676747676767476707474767070757475F9
:00000001FF
